:020000000140BD
:05000B00020054014059
:20004000758146758901D2AFD2A9D28C12005A12001B80FB438CDC0508327400F527F52662
:2000600074FFF5B0F59074FFF50DF50CF50BF50A740075F000F51A85F01BF51885F019F566
:200080001685F017F51485F0157400F513F511F525F524F523F5227400F510F50F7400F561
:2000A0002CF52B7400F51CE50860030200B10200A77400F50812030D1200CB12044B120BD5
:2000C00056120A37120AA20200A722E52104F52175F0007B647C00120E4145F07003020003
:2000E000F47400F5211200F512018112020D12028D120B0D22E50A120D907BFF120D871209
:200100000E1E45F07003020170E50A120D907B00120D87120E1E45F0700302015B7400F52C
:200120001C7400F52BE5264402F526D294E5148515F0120DFEF51485F0157B3C7C00120EB7
:200140004145F07003020158740075F000F51485F015E50A14F50A0402016DC2947401F5B9
:200160002BE52654FDF526E52754FEF527020180E52654FDF526E52754FEF5277400F52B5B
:2001800022E50B120D907BFF120D87120E1E45F070030201FCE50B120D907B00120D8712C7
:2001A0000E1E45F070030201E77400F51C7400F52CE5264408F526D293E5168517F0120DEA
:2001C000FEF51685F0177B3C7C00120E4145F070030201E4740075F000F51685F017E50B07
:2001E00014F50B040201F9C2937401F52CE52654F7F526E52754FDF52702020CE52654F7B0
:20020000F526E52754FDF5277400F52C22E50C120D907BFF120D87120E1E45F070030202E9
:2002200080E50C120D907B00120D87120E1E45F0700302026F7400F51CE5264410F526D253
:2002400092E5188519F0120DFEF51885F0197B107C0E120E4145F0700302026C740075F062
:2002600000F51885F019E50C14F50C0402027DC292E52654EFF526E52754FBF52702028C94
:20028000E52654EFF526E52754FBF52722E50D120D907BFF120D87120E1E45F070030203B0
:2002A00000E50D120D907B00120D87120E1E45F070030202EF7400F51CE5264420F526D2C2
:2002C00091E51A851BF0120DFEF51A85F01B7B107C0E120E4145F070030202EC740075F05B
:2002E00000F51A85F01BE50D14F50D040202FDC291E52654DFF526E52754F7F52702030C22
:20030000E52654DFF526E52754F7F52722E526540175F0007B007C00120E1545F070030254
:20032000044AE5B0540475F0007B007C00120E1545F0700302036CE5264401F526E52275F1
:20034000F0007B097C00120E4145F070030203547400F522E52204F52214797B7A0E75F0A9
:2003600000120D8089828A83E493F50AE5B0540875F0007B007C00120E1545F07003020321
:20038000B6E5264401F526E52375F0007B097C00120E4145F0700302039E7400F523E5238F
:2003A00004F5231479847A0E75F000120D8089828A83E493F50BE5B0541075F0007B007CA0
:2003C00000120E1545F07003020400E5264401F526E52475F0007B0D7C00120E4145F07057
:2003E000030203E87400F524E52404F52414798D7A0E75F000120D8089828A83E493F50C24
:20040000E5B0542075F0007B007C00120E1545F0700302044AE5264401F526E52575F00070
:200420007B087C00120E4145F070030204327400F525E52504F52514799A7A0E75F00012A0
:200440000D8089828A83E493F50D22E5B0543C75F0007B3C7C00120E1545F0700302046656
:20046000E52654FEF52622E509120D907B32120D87120E1545F070030204AAE52375F000F8
:200480007B087C00120E4145F070030204927400F523E52304F5231479847A0E75F00012FC
:2004A0000D8089828A83E493F50B22E51D04F51DE51D75F0007B147C00120E4145F070036B
:2004C0000204C9E52754FEF527E51D75F0007B647C00120E4145F070030204E6E5274401CB
:2004E000F5277400F51D22E51E04F51EE51E75F0007B147C00120E4145F07003020505E5B1
:200500002754FDF527E51E75F0007B647C00120E4145F07003020522E5274402F527740070
:20052000F51E22E51F04F51FE51F75F0007B147C00120E4145F07003020541E52754FBF555
:2005400027E51F75F0007BC87C00120E4145F0700302055EE5274404F5277400F51F22E5DF
:200560002004F520E52075F0007B147C00120E4145F0700302057DE52754F7F527E5207553
:20058000F0007BC87C00120E4145F0700302059AE5274408F5277400F52022E52654027012
:2005A000030205A71204ABE526540870030205B31204E7E526541070030205BF120523E571
:2005C00026542070030205CB12055F22E50D120D907BFF120D87120E1E45F0700302066D88
:2005E000740775F000792F7A00120D80C001C002E50D120D907B0A120D87120DA079717AE8
:200600000E120D8089828A83E493D007D000F6740675F000792F7A00120D80C001C002E5F9
:200620000D120D907B0A120D87120D9979717A0E120D8089828A83E493D007D000F6E527D2
:200640005408700302065A740675F000792F7A00120D80E74480F702066A740675F000795D
:200660002F7A00120D80E7547FF7020691740775F000792F7A00120D80C001C002740675D5
:20068000F000792F7A00120D807401F7D007D000F6E50C120D907BFF120D87120E1E45F06D
:2006A0007003020732740575F000792F7A00120D80C001C002E50C120D907B0A120D87128D
:2006C0000DA079717A0E120D8089828A83E493D007D000F6740475F000792F7A00120D8092
:2006E000C001C002E50C120D907B0A120D87120D9979717A0E120D8089828A83E493D0077D
:20070000D000F6E5275404700302071F740475F000792F7A00120D80E74480F702072F7428
:200720000475F000792F7A00120D80E7547FF7020756740575F000792F7A00120D80C0011F
:20074000C002740475F000792F7A00120D807401F7D007D000F6E50B120D907BFF120D8771
:20076000120E1E45F070030207F7740375F000792F7A00120D80C001C002E50B120D907B59
:200780000A120D87120DA079717A0E120D8089828A83E493D007D000F6740275F000792F2A
:2007A0007A00120D80C001C002E50B120D907B0A120D87120D9979717A0E120D8089828A75
:2007C00083E493D007D000F6E527540270030207E4740275F000792F7A00120D80E7448079
:2007E000F70207F4740275F000792F7A00120D80E7547FF7020815740375F000792F7A009B
:20080000120D807401F7740275F000792F7A00120D807401F7E50A120D907BFF120D8712F5
:200820000E1E45F070030208B6740175F000792F7A00120D80C001C002E50A120D907B0AE3
:20084000120D87120DA079717A0E120D8089828A83E493D007D000F6740075F000792F7AFB
:2008600000120D80C001C002E50A120D907B0A120D87120D9979717A0E120D8089828A83AC
:20088000E493D007D000F6E527540170030208A3740075F000792F7A00120D80E74480F787
:2008A0000208B3740075F000792F7A00120D80E7547FF70208D4740175F000792F7A001244
:2008C0000D807401F7740075F000792F7A00120D807401F71208D822740175F000792F7A09
:2008E00000120D80E775F0007B7E7C00120E1545F07003020905740175F000792F7A00129D
:200900000D807400F7740375F000792F7A00120D80E775F0007B7E7C00120E1545F07003A4
:20092000020932740375F000792F7A00120D807400F7740575F000792F7A00120D80E77577
:20094000F0007B7E7C00120E1545F0700302095F740575F000792F7A00120D807400F7746D
:200960000775F000792F7A00120D80E775F0007B7E7C00120E1545F0700302098C74077525
:20098000F000792F7A00120D807400F72278FB120D5EE6700302099DC2B002099FD2B02268
:2009A00078FB120D5EE670030209B0C2B10209B2D2B122E50E14F50E04E50E120D907B0033
:2009C000120D87120E1545F070030209F4E5112402F511E511120D9078FB120D5E86031243
:2009E0000D87120E1545F070030209F07400F5117400F50F22E51214F51204E512120D90BB
:200A00007B00120D87120E1545F07003020A36E5132402F513E513120D9078FB120D5E8653
:200A200003120D87120E1545F07003020A327400F5137400F51022E52B7003020A9FE50FB9
:200A4000120D907B00120D87120E1545F07003020A8CE51179697A0E120D90120D80898298
:200A60008A83E49375F000C0E0C0F012098D15811581E511240179697A0E120D90120D8096
:200A800089828A83E493F50E7401F50F740475F000C0E0C0F01209B315811581020AA1D2A5
:200AA000B022E52C7003020B0AE510120D907B00120D87120E1545F07003020AF7E51379B3
:200AC0006D7A0E120D90120D8089828A83E49375F000C0E0C0F01209A015811581E513248C
:200AE00001796D7A0E120D90120D8089828A83E493F5127401F510740475F000C0E0C0F0FC
:200B00001209F515811581020B0CD2B122E50A550B550C550D120D907BFF120D87120E15C5
:200B200045F07003020B55E51C04F51C14E51C75F0007B0A7C00120E4145F07003020B55AF
:200B4000740075F00CC0E0C0F0120CCC15811581C2AF758702221205CC12059B120B602285
:200B6000120D0D740075F000792F7A00120D80E775F000F54185F042E5418542F04400C590
:200B8000F04401C5F0C0E0C0F0120CCC15811581740175F000792F7A00120D80E775F0001E
:200BA000F54185F042E5418542F04400C5F04402C5F0C0E0C0F0120CCC1581158174027526
:200BC000F000792F7A00120D80E775F000F54185F042E5418542F04400C5F04403C5F0C099
:200BE000E0C0F0120CCC15811581740375F000792F7A00120D80E775F000F54185F042E594
:200C0000418542F04400C5F04404C5F0C0E0C0F0120CCC15811581740475F000792F7A0081
:200C2000120D80E775F000F54185F042E5418542F04400C5F04405C5F0C0E0C0F0120CCCCE
:200C400015811581740575F000792F7A00120D80E775F000F54185F042E5418542F044006F
:200C6000C5F04406C5F0C0E0C0F0120CCC15811581740675F000792F7A00120D80E775F06E
:200C800000F54185F042E5418542F04400C5F04407C5F0C0E0C0F0120CCC158115817407B0
:200CA00075F000792F7A00120D80E775F000F54185F042E5418542F04400C5F04408C5F0FE
:200CC000C0E0C0F0120CCC158115812278FB120D5EE60886F0F54185F042C002C0E0C0D059
:200CE000C3C297C2957A08E542339296D29700C297DAF67A08E541339296D29700C297DA4C
:200D0000F6D29500C295D0D0D0E0D00222740575F00AC0E0C0F0120CCC158115817407759D
:200D2000F00BC0E0C0F0120CCC15811581740075F009C0E0C0F0120CCC1581158174017520
:200D4000F00CC0E0C0F0120CCC15811581740075F00FC0E0C0F0120CCC1581158122C825D4
:200D600081C822C92581C97A0022D083D082CF2581F581CFC082C08322CF2581F581CF2252
:200D800029F9E5F03AFA227C00CB30E7011CCB2275F00030E70215F022120DC88EF0ED2285
:200DA000C0F0C0E0E5F06C5480FF8CF030F707EB120E0BACF0FBD0E0D0F030F703120E0BB3
:200DC000BF8005120DC88043C002C001AAF0F97E007D007F11C3E933F9EA33FADF08F5F0C9
:200DE000E9D001D00222ED33FDEE33FEC3ED9BF5F0EE9C40E0ADF0FED380DB120DFE0470D5
:200E00000205F02214B4FF0215F022120E04F4C5F0F4C5F022120E486009E4F5F022120E55
:200E20004860F7E4F5F00422120E4840F680EB120E4840EF70E480EB120E4840DD70E4806C
:200E4000D9120E4850DD80D2C5F0C39C7003E5F09B22FBE493CB22FCE493FB740193CC22F6
:200E6000FAE493F9740193CA2201140064011400147E306D79335B5F707F7BFF0003050A76
:200E80000F14191EFF0003050A0F14191EFF000102030508090A0B0C0D0EFF000102030A27
:020EA0000C0E36
:00000001FF
